:100000000C9405010C94CE110C94F5110C94FD0C7C
:100010000C94FD0C0C94FD0C0C942D010C942D01F2
:100020000C942D010C942D010C942D010C942D0198
:100030000C942D010C942D010C942D010C942D0188
:100040000C941C120C942D010C94E0140C941215B9
:100050000C942D010C942D010C942D010C942D0168
:100060000C94EB0A0C942D012020202000534154C5
:100070003D00202020200053433D00202020200070
:100080004F58434F3D002020200020414D534C3D10
:10009000004F58434F3D002031304D3D002041542A
:1000A0003D005361743D004C6F6E6720002020536B
:1000B00075727665793D0020205374617475733DC7
:1000C00000202023536174733D002020414D534C88
:1000D0003D00245245504F52542031202D312035BF
:1000E000002450524F434545440053746172746973
:1000F0006E672047505320656E67696E65004750F4
:1001000053206E6F7420726573706F6E64696E67D2
:100110000024474554504F5300537572766579203B
:10012000526571756573742053656E740024535560
:1001300052564559203100245245504F52542031D7
:10014000202D312035002450524F4345454400476F
:10015000505320436F6E74726F6C6C657200436F06
:10016000756E7420646F776E2000436F6E74726FCB
:100170006C6C6572205374617274696E6720200024
:10018000436F6E74726F6C6C65722053746172741D
:10019000696E67002A2A2050726F6772616D205362
:1001A00074617274202A2A00000000080002010015
:1001B0000003040700000000000000000102040822
:1001C00010204080010204081020010204081020C1
:1001D00004040404040404040202020202020303ED
:1001E0000303030300000000230026002900000091
:1001F0000000250028002B0000000000240027003C
:100200002A003805490A42159A0511241FBECFEF6E
:10021000D8E0DEBFCDBF11E0A0E0B1E0E8E4FCE350
:1002200002C005900D92AC3FB107D9F724E0ACEFC6
:10023000B1E001C01D92A63CB207E1F712E0C8E0B0
:10024000D2E004C02297FE010E94AA18C230D10752
:10025000C9F70E9405180C94171E0C940000809199
:100260001F029091200201969093200280931F021A
:1002700080911F0290912002039724F01092200297
:1002800010921F02089581E090E09093760280938F
:1002900075020895CF93DF93EC0166E171E085E28A
:1002A00094E00E94F415CA30D1052CF460E385E295
:1002B00094E00E94F6154AE050E0BE0185E294E029
:1002C000DF91CF910C94B616CF92DF92EF92FF920E
:1002D0000F931F93CF93DF93CDB7DEB7A8970FB6D9
:1002E000F894DEBF0FBECDBF0E947D108C010E942E
:1002F0006D10F82EE92E0E9475109C01C80164E66D
:1003000070E00E9425189F938F93EF92FF923F9386
:100310002F9388E191E09F938F937E0185E1E80E12
:10032000F11CFF92EF920E94461B0E946510D82E8E
:10033000C92E0E945D10182F092F0E945510CF92D0
:10034000DF920F931F939F938F9387E291E09F9388
:100350008F938E010F5F1F4F1F930F930E94461BB9
:1003600040E060E081EF92E00E940B11B70181EF65
:1003700092E00E94F4150FB6F894DEBF0FBECDBF19
:100380008091AD029091AE02892B31F46EE371E061
:1003900081EF92E00E94F4158091AD029091AE023F
:1003A000019731F466E371E081EF92E00E94F41569
:1003B0008091AD029091AE02029731F468E371E052
:1003C00081EF92E00E94F41580917B0290917C0273
:1003D000892BA1F460E870E081EF92E00E94C315E0
:1003E0004AE050E060917F0281EF92E00E94CB16DC
:1003F0006BE770E081EF92E00E94C31580917B0271
:1004000090917C020197B1F467E770E081EF92E090
:100410000E94C31560917702709178024AE050E023
:1004200081EF92E00E94B61662E770E081EF92E001
:100430000E94C31580917B0290917C020297A1F4E7
:100440006DE670E081EF92E00E94C3154AE050E053
:100450006091800281EF92E00E94CB1668E670E026
:1004600081EF92E00E94C31541E060E081EF92E0ED
:100470000E940B11B80181EF92E00E94F4156EE327
:1004800071E081EF92E00E94F4156FE672E081EF77
:1004900092E00E94E6156EE371E081EF92E00E9427
:1004A000F41580917B0290917C0201968330910536
:1004B0002CF490937C0280937B0204C010927C0207
:1004C00010927B02A8960FB6F894DEBF0FBECDBF88
:1004D000DF91CF911F910F91FF90EF90DF90CF9020
:1004E000089580911F0290912002892B11F40E949F
:1004F000640180911F0290912002019709F08EC043
:1005000040E060E081EF92E00E940B116AE371E04D
:1005100081EF92E00E94F4158091A9029091AA02C5
:10052000A091AB02B091AC0284369105A105B10552
:1005300030F46EE371E081EF92E00E94F415409197
:10054000A9025091AA026091AB027091AC022AE01C
:1005500030E081EF92E00E94BE1660E471E081EF2E
:1005600092E00E94F4154091990250919A02609194
:100570009B0270919C022AE030E081EF92E00E94A1
:100580006C166091910281EF92E00E94F61541E0B5
:1005900060E081EF92E00E940B1167EA70E081EF6A
:1005A00092E00E94C3158091A5029091A602A091AD
:1005B000A702B091A80284369105A105B10530F4D7
:1005C0006EE371E081EF92E00E94F4154091A50284
:1005D0005091A6026091A7027091A8022AE030E033
:1005E00081EF92E00E94BE1660E471E081EF92E03C
:1005F0000E94F415409195025091960260919702E5
:10060000709198022AE030E081EF92E00E946C162F
:1006100060918F0281EF92E00E94F61580911F0297
:1006200090912002029709F05AC040E060E081EF0B
:1006300092E00E940B1162EA70E081EF92E00E946A
:10064000C3154AE050E06091800281EF92E00E9481
:10065000CB166DE970E081EF92E00E94C3154AE08D
:1006600050E06091810281EF92E00E94CB1667E931
:1006700070E081EF92E00E94C3154AE050E0609183
:10068000820281EF92E00E94CB1641E060E081EFB0
:1006900092E00E940B1161E970E081EF92E00E940C
:1006A000C3154AE050E060917F0281EF92E00E9422
:1006B000CB166AE870E081EF92E00E94C31560916A
:1006C0008B0270918C024AE050E081EF92E00E9430
:1006D000B61666E870E081EF92E00C94C3150895B9
:1006E0004F925F926F927F928F929F92AF92BF9242
:1006F000CF92DF92EF92FF920F931F93CF93DF93EE
:10070000CDB7DEB72C970FB6F894DEBF0FBECDBFC6
:100710008091AF029091B0020E94BD1A6B017C01E2
:100720008BE6D81A85E4E80A85EFF80AC0929D02A4
:10073000D0929E02E0929F02F092A0028091B102BC
:100740009091B2020E94BD1A4B015C01E0E88E1A42
:10075000E5EB9E0AE2EAAE0AEAEFBE0A8092A10247
:100760009092A202A092A302B092A4028E010F5F07
:100770001F4F88E0F80111928A95E9F7C701B60189
:1007800020E03DE241E351E00E945B182B013C0177
:100790002F5B2983C501B40120E836E948E950E020
:1007A0000E945B1869877A878B879C872F5B2A83D7
:1007B000C301B20120E834E84EE150E00E945B182A
:1007C000205D2B8380E4482E82E4582E8FE0682E33
:1007D000712C69857A858B859C85A30192010E9485
:1007E0005B18205D2C83C701B60120E834E84EE198
:1007F00050E00E945B1825E835E441E050E00E949B
:100800005B182F592D83C501B401A30192010E94E9
:100810005B1822EC32EA40E050E00E945B182F594E
:100820002E836FEE71E08FE692E00E94AD177E019D
:10083000F7E0EF0EF11CF80161918F018FE692E075
:100840000E94F1170E151F05B1F72C960FB6F894FC
:10085000DEBF0FBECDBFDF91CF911F910F91FF90F3
:10086000EF90DF90CF90BF90AF909F908F907F9050
:100870006F905F904F9008958F929F92AF92BF922A
:10088000CF92DF92EF92FF924B015C010E946612C1
:100890006B017C01C80CD91CEA1CFB1C0E9466126F
:1008A000C616D706E806F906C8F7FF90EF90DF9066
:1008B000CF90BF90AF909F908F900895CF93DF938C
:1008C00062E082E00E942C1362E083E00E942C131D
:1008D00026E040E855E260E070E085E294E00E94A6
:1008E0007E1464EF71E080E090E00E94951240E891
:1008F00055E260E070E080E092E00E94000E64EF5C
:1009000071E080E090E00E94951264E971E085E278
:1009100094E00E94011642E050E06FE271E080E056
:100920000E94AE1142E050E063E471E081E00E9479
:10093000AE118091B9008C7F8093B9008CE08093D8
:10094000B80081EF92E00E94AB1181EF92E00E942B
:10095000AA1081EF92E00E94401181EF92E00E9484
:10096000FD1060E871E081EF92E00E94C3156AE635
:1009700071E085E294E00E94C315C8E0D0E041E058
:1009800060E081EF92E00E940B116EE571E081EF73
:1009900092E00E94C3154AE050E0BE0181EF92E070
:1009A0000E94B6166DE371E081EF92E00E94F415AB
:1009B00062E471E085E294E00E94F4154AE050E0C0
:1009C000BE0185E294E00E94B61668EE73E080E016
:1009D00090E00E943C04219791F685E294E00E9409
:1009E000FD1581EF92E00E94FD106FE471E081EF50
:1009F00092E00E94C31566E471E080E092E00E94FC
:100A0000011664EC79E080E090E00E943C0467E32A
:100A100071E080E092E00E94011640E060E081EF2A
:100A200092E00E940B1164EF71E080E090E0DF91B2
:100A3000CF910C943C046AEE70E085E294E00E9451
:100A4000011661EE70E080E092E00E9401166CEA0F
:100A50007DE080E090E00E943C0462ED70E080E088
:100A600092E00E940116E091FE01F091FF010994CD
:100A700022E040E16FE381EF92E00E9481106FEE8F
:100A800071E08FE692E00E9497176EE371E081E2D9
:100A900092E00E94971764E471E087E292E00E947E
:100AA000971768E471E08DE292E00E9497176CE47A
:100AB00071E083E392E00E94971760E571E089E3BB
:100AC00092E00E94971764E571E08FE392E00E9444
:100AD000971768E571E085E492E00E9497176CE54E
:100AE00071E08BE492E00E94971760E671E081E587
:100AF00092E00E94971764E671E087E592E00E9419
:100B0000971768E671E08DE592E00E9497176CE612
:100B100071E083E692E00E94971760E771E089E652
:100B200092E00E94971720E049E068E080E092E0C0
:100B30000C94D00DCF93DF9380E092E00E94770D6C
:100B4000CFE6D2E02697CE010E94291782E0C1327B
:100B5000D807C1F78FE692E0DF91CF910C94291767
:100B60004F925F926F927F928F929F92AF92BF92BD
:100B7000CF92DF92EF92FF92CF93DF931092B80261
:100B80001092B7021092F0028FEE91E090938A02D9
:100B90008093890282E3EEEBF2E0DF011D928A95F9
:100BA000E9F71092BD022091F002243259F14CED88
:100BB00055E060E070E080E092E00E94001741E0C4
:100BC00050E060EF72E080E092E00E9406179093A0
:100BD000BA028093B902181619067CF06EEF70E025
:100BE00085E294E00E94011681E090E09093AE02CD
:100BF0008093AD0289E090E01DC28091F002809365
:100C0000BD02D1CF81E090E09093BC028093BB0203
:100C10002093BE0280E092E00E94A60C18161906EE
:100C2000A4F480E092E00E94180C8093BD02209111
:100C3000BB023091BC02F901E254FD4F80832F5F6B
:100C40003F4F3093BC022093BB028091BD028A309B
:100C500009F7E091BB02F091BC02E354FD4F108212
:100C60006EE371E08EEB92E00E94E41A7C019093B7
:100C70008A028093890264E771E00E94F21A892B4C
:100C800029F40E941B0581E090E0D4C16CE771E07B
:100C9000C7010E94F21A892B09F04FC06EE371E080
:100CA00080E090E00E94E41A9093B4028093B30233
:100CB0000E94BD1A6093850270938602809387021A
:100CC000909388026EE371E080E090E00E94E41A65
:100CD0009093B4028093B3020E949F1A809384027F
:100CE0006EE371E080E090E00E94E41A9093B40219
:100CF0008093B3020E949F1A8093830260918502C1
:100D00007091860280918702909188026058724C9F
:100D10008A429D4E20918402621B710981099109CA
:100D20006093850270938602809387029093880275
:100D30000E94930F82E090E07DC163E871E0C701FB
:100D40000E94F21A892B09F04BC06EE371E080E03B
:100D500090E00E94E41A9093B4028093B3020E9440
:100D60009F1A809382026EE371E080E090E00E941F
:100D7000E41A9093B4028093B3026EE371E080E0D2
:100D800090E00E94E41A9093B4028093B3020E9410
:100D90009F1A809381026EE371E080E090E00E94F0
:100DA000E41A9093B4028093B3026EE371E080E0A2
:100DB00090E00E94E41A9093B4028093B3026EE331
:100DC00071E080E090E00E94E41A9093B402809376
:100DD000B3020E949F1A80937F0283E090E02AC1B1
:100DE0006BE871E0C7010E94F21A892BF1F46EE3FF
:100DF00071E080E090E00E94E41A9093B402809346
:100E0000B3020E949F1A90937A02809379026EE354
:100E100071E080E090E00E94E41A9093B402809325
:100E2000B3020E949F1A8093800266E971E080916C
:100E3000890290918A020E94F21A892BC1F56EE311
:100E400071E080E090E00E94E41A9093B4028093F5
:100E5000B3026EE371E080E090E00E94E41A9093A8
:100E6000B4028093B3026EE371E080E090E00E94F0
:100E7000E41A9093B4028093B3026EE371E080E0D1
:100E800090E00E94E41A9093B4028093B3026EE360
:100E900071E080E090E00E94E41A9093B4028093A5
:100EA000B3020E949F1A90937802809377026EE9B2
:100EB00071E08091890290918A020E94F21A892B36
:100EC00009F0B6C06EE371E080E090E00E94E41AA1
:100ED0009093B2028093B1026EE371E080E090E003
:100EE0000E94E41A9093B0028093AF026EE371E027
:100EF00080E090E00E94E41A90938E0280938D022D
:100F00000E949F1A90938C0280938B020E94700320
:100F1000E091B102F091B2028081809393028D3210
:100F200049F483E5809391023196F093B202E09305
:100F3000B10203C08EE480939102E091AF02F09180
:100F4000B0028081809393028D3249F487E58093CB
:100F50008F023196F093B002E093AF0203C085E4B4
:100F600080938F02C090B102D090B202C6010E945D
:100F7000BD1A20E4822E22E4922E2FE0A22EB12C64
:100F8000A50194010E945B1829013A012093A9024E
:100F90003093AA024093AB025093AC02C091AF02CF
:100FA000D091B002CE010E94BD1AA50194010E9409
:100FB0005B1849015A012093A5023093A602409381
:100FC000A7025093A802C6010E94BD1A6B017C01C2
:100FD000A301920160E472E48FE090E00E94151892
:100FE000C61AD70AE80AF90AC0929902D0929A0260
:100FF000E0929B02F0929C02CE010E94BD1A6B010E
:101000007C01A501940160E472E48FE090E00E940D
:101010001518C61AD70AE80AF90AC0929502D092A2
:101020009602E0929702F092980284E090E002C06B
:1010300080E090E0DF91CF91FF90EF90DF90CF9034
:10104000BF90AF909F908F907F906F905F904F90E8
:1010500008950E94751026E0289FB001299F700D09
:1010600011246F5D7D4F85E294E00E94E6156EE3EA
:1010700071E085E294E00E94F4150E946D104AE050
:1010800050E0BC0185E294E00E94B61666EA71E089
:1010900085E294E00E94F4150E947D104AE050E041
:1010A000BC0185E294E00E94B6166EE371E085E231
:1010B00094E00E94F4150E9455104AE050E0BC01F3
:1010C00085E294E00E94B6160E945D100E944A01DB
:1010D0000E9465100E944A016DE371E085E294E090
:1010E0000E94F4156FE672E085E294E00E94E61536
:1010F0006DE371E085E294E00E94F4154091A9024D
:101100005091AA026091AB027091AC022AE030E0EB
:1011100085E294E00E94BE1660E471E085E294E00E
:101120000E94F4154091990250919A0260919B029D
:1011300070919C022AE030E085E294E00E946C16F7
:101140006091910285E294E00E94F6156DE371E0F2
:1011500085E294E00E94F4154091A5025091A60208
:101160006091A7027091A8022AE030E085E294E045
:101170000E94BE1660E471E085E294E00E94F415DE
:101180004091950250919602609197027091980259
:101190002AE030E085E294E00E946C1660918F02B4
:1011A00085E294E00E94F6156AEC70E085E294E036
:1011B0000E94C31560918B0270918C024AE050E04E
:1011C00085E294E00E94B61661EC70E085E294E05E
:1011D0000E94C3154AE050E06091800285E294E0ED
:1011E0000E94CB1667EB70E085E294E00E94C31585
:1011F0004AE050E060917F0285E294E00E94CB16C5
:1012000080917702909178021816190684F46DEA9D
:1012100070E085E294E00E94C315609177027091BE
:1012200078024AE050E085E294E00E94B61685E23A
:1012300094E00E94FD1585E294E00C94F713CF939F
:10124000DF931092AE021092AD020E94B00590930F
:10125000B8028093B702C0917D02D0917E020E94B5
:101260006510C817D907A9F00E947D108A3D9740E4
:1012700034F482E090E09093AE028093AD020E943D
:1012800029080E9471020E94651090937E0280934B
:101290007D02809180028430E0F08091750290910F
:1012A00076020197B1F46DE271E080E092E00E9475
:1012B000011669E171E085E294E00E94011664E69E
:1012C00070E080E090E00E943C0410927602109260
:1012D00075020E94651065E070E00E9425189093E9
:1012E000B6028093B502892B81F461E171E080E060
:1012F00092E00E94011680E092E00E948B0C0E9416
:10130000B0059093B8028093B702DF91CF91089512
:1013100080912D0390E020912E03821B9109089566
:1013200020912E0380912D03281750F4E22FF0E036
:10133000E15DFC4F808190E02F5F20932E030895A4
:101340008FEF9FEF0895E0912E0380912D03E81712
:1013500030F4F0E0E15DFC4F808190E008958FEF84
:101360009FEF08950895CF92DF92EF92FF920F932F
:101370001F93CF93DF937C01CB018A012091090356
:10138000222389F0EB016B01C40ED51ECC15DD05BF
:1013900069F06991D701ED91FC910190F081E02D08
:1013A000C7010995F3CF642F0E94C20AC801DF91DB
:1013B000CF911F910F91FF90EF90DF90CF90089504
:1013C000CF93DF931F92CDB7DEB7698320910903D6
:1013D0002223D1F020910A03203240F021E030E0B6
:1013E000FC013383228380E090E015C080910B03E1
:1013F000E82FF0E0E45FFC4F998190838F5F80934A
:101400000B0380930A0305C061E0CE0101960E94A0
:10141000C20A81E090E00F90DF91CF910895FC0126
:101420001382128248EE53E060E070E044835583FB
:10143000668377838DEA91E091838083089510928B
:101440002E0310922D0310920B0310920A030C949A
:101450004D0A81E08093090360932C0310920B03E3
:1014600010920A0308950F93062F21E040910A037A
:101470006CE073E080912C030E946B0A10920B03C6
:1014800010920A03109209030F91089561E00C94E1
:10149000330A8DEF92E00C940F0A1092BC0381E0A6
:1014A0008093BA031092B90361E082E10E94651350
:1014B00061E083E10E946513E9EBF0E080818E7FBB
:1014C000808380818D7F808388E48093B80085E469
:1014D0008093BC0008950F93413208F04AC0909168
:1014E000BC039111FCCF92E09093BC030093BA032C
:1014F0009FEF90934F031092940340939303FB014B
:1015000065E973E0DB019A2F961B941718F491910B
:101510009D93F9CF1092BB039091BB03880F892B49
:101520008093BB038091B903813061F41092B903B9
:101530008091BB038093BB008091BC0083FDF8CFFA
:1015400085EC01C085EE8093BC00222321F08091C0
:10155000BC038230E1F380914F038F3F61F08091B3
:101560004F03803251F080914F03803341F483E088
:1015700007C081E005C080E003C082E001C084E0D4
:101580000F910895613298F42091BC03243089F4BE
:1015900060937103FC0183E793E0DC012A2F281B91
:1015A000261718F421912D93F9CF80E0089581E05A
:1015B000089582E0089585ED8093BC008091BC0081
:1015C00084FDFCCF1092BC03089585EC8093BC0091
:1015D0001092BC0308951F920F920FB60F92112420
:1015E0002F933F934F935F936F937F938F939F932B
:1015F000AF93BF93EF93FF938091B900887F8036BC
:1016000009F49EC078F5883209F45DC090F4803109
:1016100009F456C038F4882309F4F5C0883009F479
:101620004FC0F5C0883109F44EC0803209F45FC064
:10163000EEC0803409F46AC058F4803309F457C00E
:10164000883309F0E4C080934F030E94E50ADFC0AD
:10165000803509F44FC0883509F45DC0883409F03D
:10166000D6C0D3C0883909F4C4C0A8F4883709F4B7
:1016700067C038F4883609F463C0803709F460C065
:10168000C6C0883809F4B5C0803909F45FC0803815
:1016900009F0BDC05BC0803B09F483C038F4803AD8
:1016A00009F466C0883A09F47CC0B1C0803C09F4F2
:1016B000A4C0883C09F4A1C0883B09F487C0A7C036
:1016C0008091BB0310C0909194038091930398176D
:1016D00070F5E091940381E08E0F80939403F0E025
:1016E000EB56FC4F80818093BB0085EC83C08093D8
:1016F0004F038BC0E091940381E08E0F809394039D
:101700008091BB00F0E0EB56FC4F808390919403F6
:10171000809193036BC0E091940381E08E0F8093DE
:1017200094038091BB00F0E0EB56FC4F80838091E6
:10173000BA0381116AC081E08093B90384EA5EC074
:1017400083E08093BC0310925003CFCF809150036D
:10175000803208F04EC0E091500381E08E0F8093FC
:1017600050038091BB00F0E0EF5AFC4F8083BDCF67
:101770000E94E50A80915003803230F4E0915003DA
:10178000F0E0EF5AFC4F10826091500370E0E0915E
:10179000B503F091B60381E593E0099510925003EB
:1017A00036C084E08093BC031092720310927103E0
:1017B000E091B703F091B80309958091710381110D
:1017C00005C081E08093710310927303E09172036E
:1017D00081E08E0F80937203F0E0ED58FC4F808122
:1017E0008093BB009091720380917103981708F465
:1017F0007CCF85E88093BC000AC085EC8093BC0058
:101800001092BC0304C010924F030E94DB0AFF91A8
:10181000EF91BF91AF919F918F917F916F915F9168
:101820004F913F912F910F900FBE0F901F901895E1
:101830002091FF033091000428173907B9F49091E3
:10184000BD038091BE03981789F0E091BD03F0E0DD
:10185000E154FC4F80812091BD0330E02F5F3F4F6A
:101860002F7333272093BD0390E008958FEF9FEFF0
:1018700008951F93CF93DF93DC015C968D919C912B
:101880005D97009749F481E090E013969C938E93C6
:10189000129780E090E03BC05196ED91FC915297F9
:1018A00050962C915097322F30951FB75E964C91E1
:1018B0005E9741FB772770F941FD6095F894408170
:1018C000772311F0422B01C043234083EC01219781
:1018D000F1F748E0508160FF02C0522B01C0532352
:1018E0005083EC012197F1F76695415099F780817B
:1018F000772311F0832301C0822B80831FBF5C9666
:101900008D919C915D970197F1F781E090E0DF91D7
:10191000CF911F91089508952091FF033091000405
:101920002817390781F49091BD038091BE03981761
:1019300051F0E091BD03F0E0E154FC4F8081992724
:1019400087FD909508958FEF9FEF08952091FF03F5
:10195000309100042817390771F48091BE0320915B
:10196000BD0390E0805C9F4F821B910960E470E0B2
:101970000E942518089580E090E00895E091FF030B
:10198000F0910004E817F90769F4A389B4899C91E0
:101990008589809589238C93109200041092FF030F
:1019A00081E0089580E00895CF93DF93EC018A8D64
:1019B0009B8D892BF1F08091FF03909100048C178F
:1019C0009D07B9F0009711F00E94BE0C8E8D8E7F9E
:1019D0008E8F1092BE031092BD03D0930004C0936B
:1019E000FF03EB89FC8980819D89892B808381E0BD
:1019F00001C080E0DF91CF9108951F920F920FB642
:101A00000F9211242F933F934F935F936F937F9384
:101A10008F939F93AF93BF93EF93FF93E091FF0357
:101A2000F0910004309709F451C0868DA685B785E2
:101A3000958581FF04C08C91892329F447C08C913E
:101A4000892309F043C0A389B4899C918589809535
:101A500089238C93868997890197F1F7208D318DA1
:101A6000A685B785758558E040E0C9010197F1F773
:101A7000842F90E095958795482F6C91672309F006
:101A80004068515091F7868D81FD40958091BE034D
:101A900090E001968F7399272091BD03281749F094
:101AA000A091BE03B0E0A154BC4F4C938093BE0301
:101AB00003C0868D8160868F828D938D0197F1F7AB
:101AC000A389B4898C919589892B8C93FF91EF918F
:101AD000BF91AF919F918F917F916F915F914F9146
:101AE0003F912F910F900FBE0F901F9018952DEBE7
:101AF00031E0FC01318320830C94BE0C1F93CF9303
:101B0000DF93EC01162F6E8D6695617081E068277A
:101B1000812F0E94651361E0812F0E942C13812F79
:101B200090E0FC01E454FE4FE491E88BFC01E053AB
:101B3000FE4FE491F0E0EE0FFF1FE251FE4F859162
:101B400094919A8B898BDF91CF911F9108951F9368
:101B5000CF93DF93EC01162F60E0812F0E942C13AE
:101B60008E8D81FD04C061E0812F0E9465131C876A
:101B7000812F90E0FC01E454FE4FE491ED87FC01DD
:101B8000E053FE4FE491F0E0EE0FFF1FEC51FE4FEB
:101B9000859194919F878E87DF91CF911F910895B2
:101BA000FF920F931F93CF93DF93EC01F62E522FEA
:101BB0001B821A8208EE13E020E030E00C831D83C4
:101BC0002E833F838DEB91E0998388831F8A1E8A41
:101BD000198E188E1B8E1A8E1D8E1C8E8E8D8E7FEA
:101BE00050FB81F98E8F642FCE010E947E0D6F2DE8
:101BF000CE01DF91CF911F910F91FF900C94A70D13
:101C0000CF93DF93EC019A01AB011B8E1A8E198ED4
:101C1000188E1F8A1E8A60E079E08DE390E00E94B2
:101C20005B18C9012430310520F0B90163507109F6
:101C300002C061E070E07D8F6C8FEC85E63108F0CA
:101C400068C0B901769567956431710518F06351E4
:101C5000710902C061E070E07F8B6E8B069718F00F
:101C6000C901059702C081E090E0998F888FC90172
:101C7000880F991F820F931F969587959695879544
:101C80008D30910510F00C9702C081E090E09B8FA1
:101C90008A8F20916800E83050F091E0EE3008F42F
:101CA00090E081E001C0880F9A95EAF701C084E0D6
:101CB000822B809368002C85283038F02E3040F03D
:101CC000263148F48CE690E008C08DE690E005C02F
:101CD0008BE690E002C080E090E09C8B8B8B2830FC
:101CE00030F481E001C0880F2A95EAF70DC0822FF9
:101CF00090E02E3010F4089701C00E9791E001C0DB
:101D0000990F8A95EAF7892F8D8B8C8D9D8D019780
:101D1000F1F7CE01DF91CF910C94D40C6F927F92AA
:101D20008F929F92AF92BF92CF92DF92EF92FF92EB
:101D30000F931F93CF93DF93EA012CE3C22ED12C94
:101D4000E12CF12CA70196010E9439186883CA0181
:101D5000B901A70196010E9439186983CA01B90126
:101D600028E130E040E050E00E94391849015A0172
:101D70006A83CA01B9016C5F7F4F8F4F9F4F27E085
:101D800030E040E050E00E9439186F5F6B8300E064
:101D900010E0980140E054E6652E712C60E9C62EF3
:101DA000DD24D394E42FF0E0EE54F84F7F0183E07C
:101DB000E822FF24E114F10489F4CF01B3010E9469
:101DC0002518892B29F08EE691E0A0E0B0E00AC04A
:101DD000CF01B6010E942518892BA9F38DE691E069
:101DE000A0E0B0E0080F191F2A1F3B1FD901C8014E
:101DF000AA27BB2788169906AA06BB0610F04F5FD4
:101E0000D1CF4E83E114F10499F4CF0164E670E080
:101E10000E942518892B29F08EE691E0A0E0B0E021
:101E20000BC0CF0160E971E00E942518892BA1F356
:101E30008DE691E0A0E0B0E0081B190B2A0B3B0BEC
:101E4000801A910AA20AB30ACF0164E670E00E94E8
:101E500025189C01CF0160E971E00E942518E9EC8A
:101E6000F1E0A0E0A13059F4E114F10451F421159E
:101E7000310511F04DE106C00097E1F302C0408149
:101E800001C04CE150E060E070E084169506A606C3
:101E9000B70640F0841A950AA60AB70AAF5F3196D2
:101EA000AC3001F7AF5FAD8383948C82DF91CF912B
:101EB0001F910F91FF90EF90DF90CF90BF90AF9068
:101EC0009F908F907F906F900895CF92DF92EF92C6
:101ED000FF926B017C018091110490911204A091FA
:101EE0001304B0911404C816D906EA06FB0671F073
:101EF00045E154E0C701B6010E948E0EC092110464
:101F0000D0921204E0921304F0921404FF90EF9028
:101F1000DF90CF9008950E94650F80911B0490E0A0
:101F20008E54984F08950F931F9360930D047093F0
:101F30000E0480930F0490931004009106011091F9
:101F400007012091080130910901060F171F281F72
:101F5000391F00930504109306042093070430935F
:101F6000080482E090E090930404809303040E94AC
:101F700066126093090470930A0480930B04909393
:101F80000C041F910F910895CF92DF92EF92FF9270
:101F90000F931F930E946612C0900904D0900A0408
:101FA000E0900B04F0900C046C197D098E099F09D8
:101FB00000910D0410910E0420910F043091100433
:101FC000683E734081059105D8F00F5F1F4F2F4F7A
:101FD0003F4F00930D0410930E0420930F04309391
:101FE000100448EEC40E43E0D41EE11CF11CC09264
:101FF0000904D0920A04E0920B04F0920C04CACFB8
:102000008091050490910604A0910704B091080402
:10201000081719072A073B07C8F1E0910104F0915E
:102020000204309799F109956115710581059105B3
:1020300019F00E94930F2AC0809106019091070128
:10204000A0910801B091090140910D0450910E0436
:1020500060910F0470911004840F951FA61FB71F85
:102060008093050490930604A0930704B09308049A
:1020700081E090E02091030430910404232B11F4BB
:1020800080E090E0909304048093030460910D0439
:1020900070910E0480910F04909110041F910F9184
:1020A000FF90EF90DF90CF9008950E94C40F0E94A0
:1020B000650F8091170490E008950E94C40F0E945C
:1020C000650F8091160490E008950E94C40F0E944D
:1020D000650F8091150490E008950E94C40F0E943E
:1020E000650F8091190490E008950E94C40F0E942A
:1020F000650F80911A0490E008950E94C40F0C941B
:102100008B0FFC011382128289ED91E09183808311
:10211000648341872287138608951F93CF93DF93AB
:10212000EC01162F6C818DEF92E00E94290AE0915C
:10213000FD02F091FE026B85612B0190F081E02D94
:102140008DEF92E009958DEF92E0DF91CF911F9195
:102150000C94460A28E0FC01238760E00C948D1063
:102160001F93CF93DF93EC01162F64600E948D10B4
:1021700081E090E00E94BD12612F6B7FCE010E9432
:102180008D1082E390E0DF91CF911F910C94BD12EE
:102190001F93CF93DF93EC01162F0E948D10612FB8
:1021A000CE01DF91CF911F910C94B010EF92FF926E
:1021B0001F93CF93DF931F92CDB7DEB77C01162F0D
:1021C000607F642B49830E94C81080E1189FB00192
:1021D00011244981642BC7010F90DF91CF911F918A
:1021E000FF90EF900C94C81041E00E94D61081E05F
:1021F00090E0089540E00C94D61061E00E94FA103F
:1022000080ED97E00C94BD1262E00E94FA1080ED20
:1022100097E00C94BD12CF93DF93CDB7DEB728972C
:102220000FB6F894DEBF0FBECDBF28E0EEE0F1E0C0
:10223000DE01119601900D922A95E1F7FC012085AF
:10224000241710F44FEF420FFE013196E40FF11DF9
:10225000E40FF11D2081260F2068622F28960FB60B
:10226000F894DEBF0FBECDBFDF91CF910C94FA1072
:10227000FC016681262F246026836C600C94FA1082
:10228000FC0166816D7F668368600C94FA10CF93C1
:10229000DF93EC01423018F08D8188608D83488790
:1022A000222329F0413019F48D8184608D8362E30B
:1022B00070E080E090E00E9495126B85CE010E9454
:1022C0008D1068EE73E080E090E00E94951260E36C
:1022D000CE010E94C81084E991E10E94BD1260E322
:1022E000CE010E94C81084E991E10E94BD1260E312
:1022F000CE010E94C81086E990E00E94BD1260E203
:10230000CE010E94C8106D816062CE010E94FA1059
:1023100084E08E83CE010E943811CE010E94FD1010
:1023200082E08F8366E0CE010E94FA10CE01DF9139
:10233000CF910C940411CF93DF93EC018DEF92E0D9
:102340000E941F0A1D8220E04A856985CE01DF9127
:10235000CF910C9447110C949B1108958230E8F4AE
:10236000E82FF0E0EE0FFF1FE65FFE4F7183608302
:10237000813041F0809169008C7F842B80936900CB
:10238000E89A089580916900440F551F440F551F26
:10239000837F842B80936900E99A08951F920F929E
:1023A0000FB60F9211242F933F934F935F936F9328
:1023B0007F938F939F93AF93BF93EF93FF93E0919E
:1023C0000A01F0910B010995FF91EF91BF91AF9137
:1023D0009F918F917F916F915F914F913F912F913D
:1023E0000F900FBE0F901F9018951F920F920FB66F
:1023F0000F9211242F933F934F935F936F937F938B
:102400008F939F93AF93BF93EF93FF93E0910C0152
:10241000F0910D010995FF91EF91BF91AF919F91BF
:102420008F917F916F915F914F913F912F910F907D
:102430000FBE0F901F9018951F920F920FB60F921C
:1024400011242F933F938F939F93AF93BF938091CA
:102450001D0490911E04A0911F04B091200430919E
:102460001C0423E0230F2D3720F40196A11DB11D7C
:1024700005C026E8230F0296A11DB11D20931C0460
:1024800080931D0490931E04A0931F04B093200416
:102490008091210490912204A0912304B0912404FE
:1024A0000196A11DB11D8093210490932204A09355
:1024B0002304B0932404BF91AF919F918F913F91DA
:1024C0002F910F900FBE0F901F9018952FB7F89473
:1024D00060911D0470911E0480911F04909120044E
:1024E0002FBF08953FB7F894809121049091220462
:1024F000A0912304B091240426B5A89B05C02F3FCA
:1025000019F00196A11DB11D3FBF6627782F892FB5
:102510009A2F620F711D811D911D42E0660F771F7A
:10252000881F991F4A95D1F70895CF92DF92EF92B5
:10253000FF92CF93DF936B017C010E947212EB013B
:10254000C114D104E104F10489F00E9414180E941E
:1025500072126C1B7D0B683E734090F381E0C81AC9
:10256000D108E108F108C851DC4FEACFDF91CF91E3
:10257000FF90EF90DF90CF9008958230910538F072
:10258000880F991F880F991F05970197F1F70895F4
:10259000789484B5826084BD84B5816084BD85B53E
:1025A000826085BD85B5816085BDEEE6F0E0808105
:1025B00081608083E1E8F0E0108280818260808326
:1025C000808181608083E0E8F0E0808181608083A9
:1025D000E1EBF0E0808184608083E0EBF0E08081DB
:1025E00081608083EAE7F0E080818460808380817D
:1025F0008260808380818160808380818068808325
:102600001092C1000895833081F028F4813099F050
:102610008230A1F008958730A9F08830B9F0843075
:10262000D1F4809180008F7D03C0809180008F77EE
:1026300080938000089584B58F7702C084B58F7D24
:1026400084BD08958091B0008F7703C08091B00061
:102650008F7D8093B0000895CF93DF9390E0FC01CD
:10266000E454FE4F2491FC01E053FE4F84918823F3
:1026700049F190E0880F991FFC01E850FE4FA591A9
:10268000B49182519E4FFC01C591D4919FB76111C5
:1026900008C0F8948C91209582238C9388818223A2
:1026A0000AC0623051F4F8948C91322F3095832314
:1026B0008C938881822B888304C0F8948C91822B20
:1026C0008C939FBFDF91CF9108950F931F93CF936A
:1026D000DF931F92CDB7DEB7282F30E0F901E85520
:1026E000FE4F8491F901E454FE4F1491F901E05337
:1026F000FE4F04910023C9F0882321F069830E94D2
:1027000003136981E02FF0E0EE0FFF1FE251FE4F4F
:10271000A591B4919FB7F8948C91611103C0109565
:10272000812301C0812B8C939FBF0F90DF91CF91AC
:102730001F910F910895FC01818D228D90E0805CA6
:102740009F4F821B91098F7399270895FC01918DEA
:10275000828D981731F0828DE80FF11D858D90E004
:1027600008958FEF9FEF0895FC01918D828D98174A
:1027700061F0828DDF01A80FB11D5D968C91928D65
:102780009F5F9F73928F90E008958FEF9FEF089562
:1027900088E395E1892B49F080E090E0892B29F0CE
:1027A0000E94381581110C9400000895FC01848D5D
:1027B000DF01A80FB11DA35ABF4F2C91848D90E06B
:1027C00001968F739927848FA689B7892C93A08946
:1027D000B1898C9180648C93938D848D981306C0FD
:1027E0000288F389E02D80818F7D80830895CF93C7
:1027F000DF93EC01888D8823C9F0EA89FB89808109
:1028000085FD05C0A889B9898C9186FD0FC00FB6DA
:1028100007FCF5CF808185FFF2CFA889B9898C911B
:1028200085FFEDCFCE010E94D613E7CFDF91CF9188
:102830000895CF92DF92FF920F931F93CF93DF9370
:102840001F92CDB7DEB76C0181E0D60158968C930C
:1028500058975B969C915B975C968C915C979813CC
:1028600007C05096ED91FC915197808185FD2EC057
:10287000F601038D10E00F5F1F4F0F731127F02E2D
:10288000F601848DF81211C00FB607FCF9CFD601FE
:102890005096ED91FC915197808185FFF1CFC60153
:1028A00069830E94D6136981EBCF838DE80FF11DF8
:1028B000E35AFF4F6083D6015B960C935B97529669
:1028C000ED91FC915397808180620CC0D6015696A1
:1028D000ED91FC91579760835096ED91FC91519743
:1028E00080818064808381E090E00F90DF91CF91C0
:1028F0001F910F91FF90DF90CF900895BF92CF92DC
:10290000DF92EF92FF92CF93DF93EC016A017B019C
:10291000B22EE889F98982E08083411581EE58075B
:1029200061057105A1F060E079E08DE390E0A70119
:1029300096010E94391821503109410951095695D3
:10294000479537952795211580E1380798F0E88954
:10295000F989108260E874E88EE190E0A7019601A1
:102960000E9439182150310941095109569547955E
:1029700037952795EC85FD853083EE85FF8520838F
:10298000188EEC89FD89B082EA89FB89808180619B
:102990008083EA89FB89808188608083EA89FB895A
:1029A000808180688083EA89FB8980818F7D808334
:1029B000DF91CF91FF90EF90DF90CF90BF9008957F
:1029C0001F920F920FB60F9211242F938F939F9304
:1029D000EF93FF93E0913504F09136048081E0910C
:1029E0003B04F0913C0482FD12C0908180913E0432
:1029F0008F5F8F7320913F04821751F0E0913E0466
:102A0000F0E0EB5DFB4F958F80933E0401C0808129
:102A1000FF91EF919F918F912F910F900FBE0F908B
:102A20001F9018951F920F920FB60F9211242F939B
:102A30003F934F935F936F937F938F939F93AF9346
:102A4000BF93EF93FF9385E294E00E94D613FF912A
:102A5000EF91BF91AF919F918F917F916F915F9116
:102A60004F913F912F910F900FBE0F901F9018958F
:102A700085E294E00E949B1321E0892B09F420E079
:102A8000822F0895109228041092270488EE93E074
:102A9000A0E0B0E08093290490932A04A0932B0433
:102AA000B0932C0481EE91E090932604809325044A
:102AB00085EC90E0909332048093310484EC90E0B4
:102AC000909334048093330480EC90E09093360428
:102AD0008093350481EC90E0909338048093370420
:102AE00082EC90E090933A048093390486EC90E075
:102AF00090933C0480933B0410923E0410923F0458
:102B000010924004109241040895CF92DF92EF9208
:102B1000FF920F931F93CF93DF937C016A01EB0128
:102B200000E010E00C151D0571F06991D701ED91E1
:102B3000FC910190F081E02DC7010995892B19F0D6
:102B40000F5F1F4FEFCFC801DF91CF911F910F9102
:102B5000FF90EF90DF90CF9008956115710581F09F
:102B6000DB010D900020E9F7AD0141505109461BF2
:102B7000570BDC01ED91FC910280F381E02D09946B
:102B800080E090E00895EF92FF920F931F93CF9310
:102B9000DF938C017B01C0E0D0E0F701EC0FFD1F5B
:102BA0006491662359F0F801A081B181ED91FC9107
:102BB000C8010995892B11F02196EFCFCE01DF9145
:102BC000CF911F910F91FF90EF900895DC01ED914F
:102BD000FC91DB0114964D915C9115976D917C9160
:102BE0000280F381E02D09940C94AD15DC01ED9188
:102BF000FC910190F081E02D09946DEE71E00C9450
:102C0000AD150F931F93CF93DF93EC010E94C31573
:102C10008C01CE010E94FD15800F911FDF91CF9195
:102C20001F910F9108958F929F92AF92BF92CF9272
:102C3000DF92EF92FF920F931F93CF93DF93CDB765
:102C4000DEB7A1970FB6F894DEBF0FBECDBF7C01F3
:102C5000C42EE52FCB01D22E19A221E02D1510F0A4
:102C60002AE0D22E8E010F5D1F4F8D2C912CA12CAE
:102C7000B12C6C2D7E2FA50194010E9439188C2D4A
:102C8000D29E80191124015011098A3014F4805DFC
:102C900001C0895CF801808321153105410551058A
:102CA00021F0C22EE32FCA01E4CFB801C7010E9470
:102CB000AD15A1960FB6F894DEBF0FBECDBFDF9164
:102CC000CF911F910F91FF90EF90DF90CF90BF9029
:102CD000AF909F908F900895CF92DF92EF92FF92E6
:102CE0000F931F93CF93DF93EC016A017B012115B2
:102CF000310579F4E881F9810190F081E02D642FAC
:102D0000DF91CF911F910F91FF90EF90DF90CF90C7
:102D100009942A303105E9F477FF1AC06DE20E9468
:102D2000F6158C0144275527BA014C195D096E0927
:102D30007F092AE0CE010E941316800F911FDF91B8
:102D4000CF911F910F91FF90EF90DF90CF9008955A
:102D50002AE0B701A601CE01DF91CF911F910F911B
:102D6000FF90EF90DF90CF900C9413169A01AB0177
:102D7000662757FD6095762F0C946C16211531054A
:102D800041F4DC01ED91FC910190F081E02D642F84
:102D900009940C9413169A01462F50E060E070E0FD
:102DA0000C94BE160F931F93CF93DF93EC010E94F8
:102DB0006612688779878A879B87E881F981068010
:102DC000F781E02DCE01099597FF15C00E9466128C
:102DD000088519852A853B85601B710B820B930B37
:102DE0000C811D812E813F81601771078207930737
:102DF00020F38FEF9FEFDF91CF911F910F910895F7
:102E0000FC0144835583668377830895CF92DF92D4
:102E1000EF92FF920F931F93CF93DF937C016A0190
:102E2000EB0100E010E00C151D0549F0C7010E9400
:102E3000D21697FD04C089930F5F1F4FF4CFC801CE
:102E4000DF91CF911F910F91FF90EF90DF90CF9086
:102E50000895FC01808191810C944619CF93DF93F2
:102E6000EC0188819981009711F00E94461919821E
:102E700018821D821C821B821A82DF91CF910895D5
:102E80000F931F93CF93DF93EC018B016F5F7F4F05
:102E9000888199810E94D519009731F099838883A0
:102EA0001B830A8381E001C080E0DF91CF911F91F5
:102EB0000F910895CF93DF93EC0188819981892B3D
:102EC00029F08A819B818617970760F4CE010E94C2
:102ED0004017882341F08C819D81892B19F4E8816A
:102EE000F981108281E0DF91CF910895EF92FF92F6
:102EF0000F931F93CF93DF93EC017B018A01BA01FB
:102F00000E945A17811104C0CE010E942E1707C0DB
:102F10001D830C83B701888199810E94FB1ACE0121
:102F2000DF91CF911F910F91FF90EF900895FC01D9
:102F3000118210821382128215821482611571052A
:102F400059F0FB0101900020E9F7AF014150510910
:102F5000461B570B0C9476170895CF93DF93EC0123
:102F60006115710561F0FB0101900020E9F7AF01E7
:102F700041505109461B570B0E94761702C00E9410
:102F80002E17CE01DF91CF910895EF92FF920F930C
:102F90001F93CF93DF93EC017B010C811D816115A1
:102FA000710511F480E016C04115510591F0040F30
:102FB000151FB8010E945A178823A1F3288139816F
:102FC0008C819D81B701820F931F0E94FB1A1D8384
:102FD0000C8381E0DF91CF911F910F91FF90EF90D3
:102FE0000895CF93DF9300D0CDB7DEB769831A82FF
:102FF00041E050E0BE016F5F7F4F0E94C5170F9008
:103000000F90DF91CF91089508950E94C8120E94F9
:1030100004180E945E04C8ECD3E10E941F092097A7
:10302000E1F30E94C813F9CF0895DB018F939F93BA
:103030000E948918BF91AF91A29F800D911DA39FFF
:10304000900DB29F900D1124089597FB072E16F452
:10305000009407D077FD09D00E94941807FC05D092
:103060003EF4909581959F4F0895709561957F4F9F
:103070000895A1E21A2EAA1BBB1BFD010DC0AA1FB9
:10308000BB1FEE1FFF1FA217B307E407F50720F0D1
:10309000A21BB30BE40BF50B661F771F881F991F4C
:1030A0001A9469F760957095809590959B01AC0195
:1030B000BD01CF010895052E97FB1EF400940E94D8
:1030C000721857FD07D00E94391807FC03D04EF440
:1030D0000C94721850954095309521953F4F4F4F65
:1030E0005F4F089590958095709561957F4F8F4FB4
:1030F0009F4F0895A29FB001B39FC001A39F700D81
:10310000811D1124911DB29F700D811D1124911DEF
:1031100008950E947A18A59F900DB49F900DA49FCA
:10312000800D911D11240895AA1BBB1B51E107C0FE
:10313000AA1FBB1FA617B70710F0A61BB70B881F47
:10314000991F5A95A9F780959095BC01CD010895D6
:10315000EE0FFF1F0590F491E02D0994CF93DF93BC
:103160008230910510F482E090E0E091C404F09187
:10317000C50420E030E0A0E0B0E0309739F14081B4
:10318000518148175907B8F04817590771F48281DF
:103190009381109729F013969C938E9312972CC0CD
:1031A0009093C5048093C40427C02115310531F0E4
:1031B0004217530718F0A901DB0101C0EF019A0182
:1031C000BD01DF010280F381E02DD7CF211531054C
:1031D000F9F0281B390B2430310580F48A819B815A
:1031E0006115710521F0FB019383828304C09093E4
:1031F000C5048093C404FE01329644C0FE01E20F70
:10320000F31F8193919322503109398328833AC067
:103210002091C2043091C304232B41F42091020178
:10322000309103013093C3042093C2042091000124
:10323000309101012115310541F42DB73EB7409180
:10324000040150910501241B350BE091C204F0915B
:10325000C304E217F307A0F42E1B3F0B281739070E
:1032600078F0AC014E5F5F4F2417350748F04E0FE2
:103270005F1F5093C3044093C2048193919302C093
:10328000E0E0F0E0CF01DF91CF910895CF93DF939D
:10329000009709F487C0FC01329713821282C09113
:1032A000C404D091C504209781F420813181280F76
:1032B000391F8091C2049091C3048217930779F556
:1032C000F093C304E093C2046DC0DE0120E030E05F
:1032D000AE17BF0750F412964D915C9113979D0164
:1032E0004115510509F1DA01F3CFB383A28340817F
:1032F0005181840F951F8A179B0771F48D919C91C2
:103300001197840F951F02969183808312968D9159
:103310009C911397938382832115310529F4F093AF
:10332000C504E093C4043EC0D9011396FC93EE9308
:1033300012974D915D91A40FB51FEA17FB0779F421
:1033400080819181840F951F0296D90111969C93DB
:103350008E938281938113969C938E931297E0E0D3
:10336000F0E08A819B81009719F0FE01EC01F9CF12
:10337000CE01029628813981820F931F2091C204C9
:103380003091C3042817390769F4309729F4109253
:10339000C5041092C40402C013821282D093C304E5
:1033A000C093C204DF91CF910895A0E0B0E0EBEDAF
:1033B000F9E10C94E41DEC01CB01209719F40E9473
:1033C000AE18B8C0FE01E60FF71F9E01225031096A
:1033D000E217F30708F4ACC0D9010D911C911197C5
:1033E00006171707B8F00530110508F49FC0A801AB
:1033F000445051094617570708F498C00250110964
:10340000061B170B019311936D937C93CF010E94C0
:1034100046198CC05B01A01AB10A4E01800E911EA4
:10342000A091C404B091C504612C712C60E070E0DF
:10343000109709F449C0A815B905C9F5ED90FC909D
:103440001197670142E0C40ED11CCA14DB0478F165
:1034500047018A189B08640142E0C40ED11C1296F1
:10346000BC9012971396AC91B5E0CB16D10440F006
:10347000B282A38391828082D9018D939C9309C0EB
:103480000E5F1F4F0E0D1F1DF90111830083EB2DE1
:10349000FA2F6115710531F0DB011396FC93EE9361
:1034A000129744C0F093C504E093C4043FC06D91EB
:1034B0007C9111976616770608F43B01BD011296C0
:1034C0000D90BC91A02DB4CF6091C2047091C30443
:1034D00068157905E9F468167906D0F44091000181
:1034E000509101014115510541F44DB75EB760910E
:1034F000040170910501461B570BE417F507C0F452
:10350000F093C304E093C204F901918380830EC059
:103510000E94AE187C01009759F0A801BE010E94DC
:10352000E91ACE010E944619C70104C0CE0102C0AB
:1035300080E090E0CDB7DEB7EEE00C94001EFC0119
:1035400088279927E89421912032E9F3293010F057
:103550002E30C8F32B3241F02D3239F4689404C078
:103560000E943E1B820F911D219120532A30C0F3EF
:103570001EF4909581959F4F08951F93FC01992704
:103580008827BC01E89411911032E9F3193010F04A
:103590001E30C8F31B3251F01D3249F4689406C046
:1035A0000E94291B610F711D811D911D11911053E6
:1035B0001A30B0F33EF490958095709561957F4FE9
:1035C0008F4F9F4F1F9108954CEF51E00E94021BB7
:1035D0000895FB01DC0102C001900D924150504062
:1035E000D8F70895FB01DC018D910190801901103D
:1035F000D9F3990B0895FB01DC0101900D92002095
:10360000E1F70895FA01A191B081009719F410979C
:10361000E1F0CD01DC01CD010D90002011F4C001DD
:1036200013C0FB012191222319F02015D9F7F3CF04
:10363000FB012191201519F41E92119606C0222338
:10364000C1F70D900020A1F7D001FA01A193B0833A
:103650000895592F482F372F262F660F771F881F61
:10366000991F660F771F881F991F620F731F841F92
:10367000951F660F771F881F991F08957AE0979FFF
:10368000902D879F802D910D11240895AEE0B0E01C
:10369000ECE4FBE10C94EE1D0D891E8986E08C8321
:1036A0001A8309838FEF9FE79E838D83AE01475E68
:1036B0005F4F6F89788DCE0101960E94681BEF8164
:1036C000F885E00FF11F10822E96E4E00C940A1E9C
:1036D000ACE0B0E0EEE6FBE10C94E01D7C016B0198
:1036E0008A01FC0117821682838181FFBDC1CE0150
:1036F00001964C01F7019381F60193FD859193FFAB
:1037000081916F01882309F4ABC1853239F493FDAF
:10371000859193FF81916F01853229F4B70190E083
:103720000E94501DE7CF512C312C20E02032A0F414
:103730008B3269F030F4803259F0833269F42061C1
:103740002CC08D3239F0803339F4216026C02260DC
:10375000246023C0286021C027FD27C030ED380F2A
:103760003A3078F426FF06C0FAE05F9E300D11244F
:10377000532E13C08AE0389E300D1124332E206260
:103780000CC08E3221F426FD6BC1206406C08C363D
:1037900011F4206802C0883641F4F60193FD85914A
:1037A00093FF81916F018111C1CF982F9F7D955417
:1037B000933028F40C5F1F4FFFE3F9830DC083366D
:1037C00031F0833771F0833509F05BC022C0F80116
:1037D000808189830E5F1F4F44244394512C5401F0
:1037E00015C03801F2E06F0E711CF801A080B180A5
:1037F00026FF03C0652D70E002C06FEF7FEFC501AB
:103800002C870E94451D2C0183012C852F77222EA9
:1038100017C03801F2E06F0E711CF801A080B18072
:1038200026FF03C0652D70E002C06FEF7FEFC5017A
:103830002C870E943A1D2C012C852068222E8301A2
:1038400023FC1BC0832D90E048165906B0F4B70145
:1038500080E290E00E94501D3A94F4CFF50127FCDD
:10386000859127FE81915F01B70190E00E94501D74
:1038700031103A94F1E04F1A51084114510471F794
:10388000E5C0843611F0893639F5F80127FF07C005
:1038900060817181828193810C5F1F4F08C06081BC
:1038A0007181882777FD8095982F0E5F1F4F2F76A7
:1038B000B22E97FF09C090958095709561957F4FC6
:1038C0008F4F9F4F2068B22E2AE030E0A4010E9463
:1038D000821DA82EA81844C0853729F42F7EB22E49
:1038E0002AE030E025C0F22FF97FBF2E8F36C1F0DD
:1038F00018F4883579F0B4C0803719F0883721F092
:10390000AFC02F2F2061B22EB4FE0DC08B2D84606E
:10391000B82E09C024FF0AC09F2F9660B92E06C09A
:1039200028E030E005C020E130E002C020E132E0D4
:10393000F801B7FE07C060817181828193810C5FBD
:103940001F4F06C06081718180E090E00E5F1F4FC5
:10395000A4010E94821DA82EA818FB2DFF77BF2E60
:10396000B6FE0BC02B2D2E7FA51450F4B4FE0AC05A
:10397000B2FC08C02B2D2E7E05C07A2C2B2D03C047
:103980007A2C01C0752C24FF0DC0FE01EA0DF11D3B
:103990008081803311F4297E09C022FF06C0739410
:1039A000739404C0822F867809F0739423FD13C0AA
:1039B00020FF06C05A2C731418F4530C5718732C9C
:1039C000731468F4B70180E290E02C870E94501DC8
:1039D00073942C85F5CF731410F4371801C0312C73
:1039E00024FF12C0B70180E390E02C870E94501D95
:1039F0002C8522FF17C021FF03C088E590E002C09C
:103A000088E790E0B7010CC0822F867859F021FD3D
:103A100002C080E201C08BE227FD8DE2B70190E099
:103A20000E94501DA51438F4B70180E390E00E9475
:103A3000501D5A94F7CFAA94F401EA0DF11D80812C
:103A4000B70190E00E94501DA110F5CF332009F47A
:103A500051CEB70180E290E00E94501D3A94F6CF1B
:103A6000F7018681978102C08FEF9FEF2C96E2E1EC
:103A70000C94FC1DFC010590615070400110D8F7BA
:103A8000809590958E0F9F1F0895FC0161507040A6
:103A900001900110D8F7809590958E0F9F1F089583
:103AA0000F931F93CF93DF93182F092FEB018B8177
:103AB00081FD03C08FEF9FEF20C082FF10C04E81B9
:103AC0005F812C813D81421753077CF4E881F981A5
:103AD0009F012F5F3F4F39832883108306C0E885FD
:103AE000F985812F0995892B29F72E813F812F5F39
:103AF0003F4F3F832E83812F902FDF91CF911F91D6
:103B00000F910895FA01AA27283051F1203181F14F
:103B1000E8946F936E7F6E5F7F4F8F4F9F4FAF4FD5
:103B2000B1E03ED0B4E03CD0670F781F891F9A1FE8
:103B3000A11D680F791F8A1F911DA11D6A0F711D9C
:103B4000811D911DA11D20D009F468943F912AE0A8
:103B5000269F11243019305D3193DEF6CF01089590
:103B6000462F4770405D4193B3E00FD0C9F7F6CFC1
:103B7000462F4F70405D4A3318F0495D31FD405289
:103B8000419302D0A9F7EACFB4E0A695979587951F
:103B900077956795BA95C9F70097610571050895FE
:103BA0009B01AC010A2E06945795479537952795AA
:103BB000BA95C9F7620F731F841F951FA01D089542
:103BC0002F923F924F925F926F927F928F929F922D
:103BD000AF92BF92CF92DF92EF92FF920F931F931B
:103BE000CF93DF93CDB7DEB7CA1BDB0B0FB6F894CC
:103BF000DEBF0FBECDBF09942A88398848885F840C
:103C00006E847D848C849B84AA84B984C884DF807C
:103C1000EE80FD800C811B81AA81B981CE0FD11D60
:103C20000FB6F894DEBF0FBECDBFED01089512E0D0
:103C3000C8E0D2E004C0FE010E94AA182296CA3051
:083C4000D107C9F7F894FFCF8A
:103C48000000C60480002C010000AD11AD11000079
:103C58004000140054003A00253032642F253032D9
:103C6800642F2530326400253032643A25303264BE
:103C78003A25303264002A003F004C61742020004D
:103C88002E002C004A616E00466562004D6172008C
:103C9800417072004D6179004A756E004A756C007A
:103CA80041756700536570004F6374004E6F76006E
:103CB80044656300244745545645520024434C4FFD
:103CC800434B0024535441545553002445585453EE
:103CD80054415455530024535552564559002447CE
:103CE8004554504F53002C200000000000E009B359
:103CF8000988099009A309B20900000000390C8558
:103D080015A60C180C8C0C8B0C1F1C1F1E1F1E1FBD
:103D18001F1E1F1E1F00000000F410851500000064
:103D280000191485159B13B413A613F7130D0A0075
:0C3D38006E616E00696E66006F766600BA
:00000001FF
